:020000040000FA
:020000000428D2
:08000800FF30A200FF30A3004D
:1000100007309F0023106820A3106720231166205B
:10002000A311652023126420A312632023136220EE
:10003000A313612022146C20A2146B2022156A20C5
:10004000A2156920A0140330A500A60125084320AD
:10005000A01C2C28A60A2F2801302602A60026085C
:100060005C20051836280530A5003A2885183A285E
:100070000130A50005193E28A01441288519412802
:10008000A01026284228A7002708A8006430A9004D
:100090000A304A28AA00FF30AB002908AD00280822
:1000A000AC0017302B0703185228AC0B5128AD0BAE
:1000B0004F28AA0B4D280800A4005E2824088600BB
:1000C00008006D286D286D286D286D286D286D2815
:1000D0006D28702870287028702823086600080092
:0600E00022086500080083
:02400E00103F61
:00000001FF
